******************************************************************************
             TMS320C2000 Linker PC v21.6.0                     
******************************************************************************
>> Linked Thu Nov 24 13:40:34 2022

OUTPUT FILE NAME:   <sdl_ex_flash_ecc_test.out>
ENTRY POINT SYMBOL: "code_start"  address: 00080000


MEMORY CONFIGURATION

         name            origin    length      used     unused   attr    fill
----------------------  --------  ---------  --------  --------  ----  --------
PAGE 0:
  RAMM0                 000000f6   0000030a  00000000  0000030a  RWIX
  RAMLS0                00008000   00000800  00000172  0000068e  RWIX
  RAMLS1                00008800   00000800  00000000  00000800  RWIX
  RAMLS2                00009000   00000800  00000000  00000800  RWIX
  RAMLS3                00009800   00000800  00000000  00000800  RWIX
  RAMLS4                0000a000   00000800  00000000  00000800  RWIX
  BEGIN                 00080000   00000002  00000002  00000000  RWIX
  FLASH_BANK0_SEC0      00080002   00000ffe  00000000  00000ffe  RWIX
  FLASH_BANK0_SEC1      00081000   00001000  0000018e  00000e72  RWIX
  FLASH_BANK0_SEC2      00082000   00001000  00000bba  00000446  RWIX
  FLASH_BANK0_SEC3      00083000   00001000  00000000  00001000  RWIX
  FLASH_BANK0_SEC4      00084000   00001000  000001fe  00000e02  RWIX
  FLASH_BANK0_SEC5      00085000   00001000  00000000  00001000  RWIX
  FLASH_BANK0_SEC6      00086000   00001000  00000000  00001000  RWIX
  FLASH_BANK0_SEC7      00087000   00001000  00000000  00001000  RWIX
  FLASH_BANK0_SEC8      00088000   00001000  00000000  00001000  RWIX
  FLASH_BANK0_SEC9      00089000   00001000  00000000  00001000  RWIX
  FLASH_BANK0_SEC10     0008a000   00001000  00000000  00001000  RWIX
  FLASH_BANK0_SEC11     0008b000   00001000  00000000  00001000  RWIX
  FLASH_BANK0_SEC12     0008c000   00001000  00000000  00001000  RWIX
  FLASH_BANK0_SEC13     0008d000   00001000  00000000  00001000  RWIX
  FLASH_BANK0_SEC14     0008e000   00001000  00000000  00001000  RWIX
  FLASH_BANK0_SEC15     0008f000   00001000  00000000  00001000  RWIX
  FLASH_BANK1_SEC0      00090000   00001000  00000000  00001000  RWIX
  FLASH_BANK1_SEC1      00091000   00001000  00000000  00001000  RWIX
  FLASH_BANK1_SEC2      00092000   00001000  00000000  00001000  RWIX
  FLASH_BANK1_SEC3      00093000   00001000  00000000  00001000  RWIX
  FLASH_BANK1_SEC4      00094000   00001000  00000000  00001000  RWIX
  FLASH_BANK1_SEC5      00095000   00001000  00000000  00001000  RWIX
  FLASH_BANK1_SEC6      00096000   00001000  00000000  00001000  RWIX
  FLASH_BANK1_SEC7      00097000   00001000  00000000  00001000  RWIX
  FLASH_BANK1_SEC8      00098000   00001000  00000000  00001000  RWIX
  FLASH_BANK1_SEC9      00099000   00001000  00000000  00001000  RWIX
  FLASH_BANK1_SEC10     0009a000   00001000  00000000  00001000  RWIX
  FLASH_BANK1_SEC11     0009b000   00001000  00000000  00001000  RWIX
  FLASH_BANK1_SEC12     0009c000   00001000  00000000  00001000  RWIX
  FLASH_BANK1_SEC13     0009d000   00001000  00000000  00001000  RWIX
  FLASH_BANK1_SEC14     0009e000   00001000  00000000  00001000  RWIX
  FLASH_BANK1_SEC15     0009f000   00000ff0  00000000  00000ff0  RWIX
  RESET                 003fffc0   00000002  00000000  00000002  RWIX

PAGE 1:
  BOOT_RSVD             00000002   000000f1  00000000  000000f1  RWIX
  RAMM1                 00000400   000003f8  00000100  000002f8  RWIX
  RAMLS5                0000a800   00000800  00000018  000007e8  RWIX
  RAMLS6                0000b000   00000800  00000000  00000800  RWIX
  RAMLS7                0000b800   00000800  00000000  00000800  RWIX
  RAMGS0                0000c000   00002000  00000000  00002000  RWIX
  RAMGS1                0000e000   00002000  00000000  00002000  RWIX
  RAMGS2                00010000   00002000  00000000  00002000  RWIX
  RAMGS3                00012000   00001ff8  00000000  00001ff8  RWIX


SECTION ALLOCATION MAP

 output                                  attributes/
section   page    origin      length       input sections
--------  ----  ----------  ----------   ----------------
codestart 
*          0    00080000    00000002     
                  00080000    00000002     f28004x_codestartbranch.obj (codestart)

.cinit     0    00081174    0000001c     
                  00081174    0000000a     (.cinit..data.load) [load image, compression = lzss]
                  0008117e    00000006     (__TI_handler_table)
                  00081184    00000004     (.cinit..bss.load) [load image, compression = zero_init]
                  00081188    00000008     (__TI_cinit_table)

.reset     0    003fffc0    00000000     DSECT

.stack     1    00000400    00000100     UNINITIALIZED
                  00000400    00000100     --HOLE--

.init_array 
*          0    00081000    00000000     UNINITIALIZED

.bss       1    0000a800    0000000c     UNINITIALIZED
                  0000a800    0000000c     sdl_ex_flash_ecc_test.obj (.bss)

.data      1    0000a80c    0000000c     UNINITIALIZED
                  0000a80c    00000006     rts2800_fpu32_eabi.lib : exit.c.obj (.data)
                  0000a812    00000002                            : _lock.c.obj (.data:_lock)
                  0000a814    00000002                            : _lock.c.obj (.data:_unlock)
                  0000a816    00000002     sdl_ex_flash_ecc_test.obj (.data)

.const     0    00084000    000001fe     
                  00084000    0000009b     driverlib_eabi.lib : flash.obj (.const:.string)
                  0008409b    00000001     --HOLE-- [fill = 0]
                  0008409c    0000009a                        : sysctl.obj (.const:.string)
                  00084136    00000098                        : gpio.obj (.const:.string)
                  000841ce    00000020     sdl_ex_flash_ecc_test.obj (.const:$P$T1$2)
                  000841ee    00000010     sdl_ex_flash_ecc_test.obj (.const:$P$T0$1)

.TI.ramfunc 
*          0    00081000    00000172     RUN ADDR = 00008000
                  00081000    00000044     driverlib_eabi.lib : flash.obj (.TI.ramfunc:Flash_initModule)
                  00081044    0000003e     sdl_ex_flash_ecc_test.obj (.TI.ramfunc:testECCBlock)
                  00081082    0000002d     driverlib_eabi.lib : flash.obj (.TI.ramfunc:Flash_setBankPowerMode)
                  000810af    00000024                        : flash.obj (.TI.ramfunc:Flash_setWaitstates)
                  000810d3    0000001e                        : flash.obj (.TI.ramfunc:Flash_setPumpPowerMode)
                  000810f1    0000001a                        : flash.obj (.TI.ramfunc:Flash_disableCache)
                  0008110b    0000001a                        : flash.obj (.TI.ramfunc:Flash_disablePrefetch)
                  00081125    00000019                        : flash.obj (.TI.ramfunc:Flash_enableCache)
                  0008113e    00000019                        : flash.obj (.TI.ramfunc:Flash_enablePrefetch)
                  00081157    00000017                        : flash.obj (.TI.ramfunc:Flash_enableECC)
                  0008116e    00000004                        : sysctl.obj (.TI.ramfunc)

.text      0    00082000    00000bba     
                  00082000    000000e0     device.obj (.text:Device_enableAllPeripherals)
                  000820e0    000000c7     driverlib_eabi.lib : sysctl.obj (.text:SysCtl_setClock)
                  000821a7    000000c0                        : sysctl.obj (.text:SysCtl_isPLLValid)
                  00082267    000000bb     sdl_ex_flash_ecc_test.obj (.text:calculateECC)
                  00082322    0000007a     driverlib_eabi.lib : sysctl.obj (.text:DCC_setCounterSeeds)
                  0008239c    0000006d     sdl_ex_flash_ecc_test.obj (.text:corrErrorISR)
                  00082409    00000060     sdl_ex_flash_ecc_test.obj (.text:runCorrectableDataErrorTest)
                  00082469    00000057     sdl_ex_flash_ecc_test.obj (.text:main)
                  000824c0    00000052     driverlib_eabi.lib : gpio.obj (.text:GPIO_setPadConfig)
                  00082512    0000004a                        : sysctl.obj (.text:SysCtl_selectOscSource)
                  0008255c    00000046     sdl_ex_flash_ecc_test.obj (.text:nmiISR)
                  000825a2    0000003e     device.obj (.text:Device_init)
                  000825e0    0000003d     driverlib_eabi.lib : interrupt.obj (.text:Interrupt_initModule)
                  0008261d    0000003b                        : gpio.obj (.text:GPIO_setAnalogMode)
                  00082658    00000039     sdl_ex_flash_ecc_test.obj (.text:runCorrectableECCErrorTest)
                  00082691    00000034     driverlib_eabi.lib : interrupt.obj (.text:Interrupt_enable)
                  000826c5    00000031                        : gpio.obj (.text:GPIO_setDirectionMode)
                  000826f6    00000031     rts2800_fpu32_eabi.lib : copy_decompress_lzss.c.obj (.text:decompress:lzss)
                  00082727    00000031     sdl_ex_flash_ecc_test.obj (.text:runUncorrectableErrorTest)
                  00082758    0000002b     rts2800_fpu32_eabi.lib : autoinit.c.obj (.text:__TI_auto_init_nobinit_nopinit)
                  00082783    00000029                            : exit.c.obj (.text)
                  000827ac    00000026     driverlib_eabi.lib : sysctl.obj (.text:SysCtl_pollX1Counter)
                  000827d2    00000025                        : sysctl.obj (.text:DCC_enableSingleShotMode)
                  000827f7    00000024                        : sysctl.obj (.text:SysCtl_selectXTAL)
                  0008281b    0000001f                        : sysctl.obj (.text:DCC_setCounter1ClkSource)
                  0008283a    0000001e                        : interrupt.obj (.text:Interrupt_initVectorTable)
                  00082858    0000001e     rts2800_fpu32_eabi.lib : ll_cmp28.asm.obj (.text)
                  00082876    0000001d     driverlib_eabi.lib : sysctl.obj (.text:DCC_setCounter0ClkSource)
                  00082893    0000001d     rts2800_fpu32_eabi.lib : memcpy.c.obj (.text)
                  000828b0    0000001a     driverlib_eabi.lib : sysctl.obj (.text:SysCtl_selectXTALSingleEnded)
                  000828ca    00000018     rts2800_fpu32_eabi.lib : ll_aox28.asm.obj (.text)
                  000828e2    00000017     driverlib_eabi.lib : sysctl.obj (.text:DCC_disableDoneSignal)
                  000828f9    00000017                        : sysctl.obj (.text:DCC_enableDoneSignal)
                  00082910    00000017     device.obj (.text:SysCtl_enablePeripheral)
                  00082927    00000017     driverlib_eabi.lib : sysctl.obj (.text:SysCtl_enablePeripheral)
                  0008293e    00000017     rts2800_fpu32_eabi.lib : boot28.asm.obj (.text)
                  00082955    00000016     driverlib_eabi.lib : sysctl.obj (.text:DCC_clearDoneFlag)
                  0008296b    00000016                        : sysctl.obj (.text:DCC_clearErrorFlag)
                  00082981    00000016                        : sysctl.obj (.text:DCC_disableErrorSignal)
                  00082997    00000016                        : sysctl.obj (.text:DCC_enableErrorSignal)
                  000829ad    00000014                        : sysctl.obj (.text:DCC_disableModule)
                  000829c1    00000014                        : sysctl.obj (.text:DCC_enableModule)
                  000829d5    00000014                        : gpio.obj (.text:GPIO_isPinValid)
                  000829e9    00000010     device.obj (.text:ASysCtl_disableDCDC)
                  000829f9    00000010     driverlib_eabi.lib : sysctl.obj (.text:DCC_isBaseValid)
                  00082a09    00000010                        : flash.obj (.text:Flash_isCtrlBaseValid)
                  00082a19    00000010                        : flash.obj (.text:Flash_isECCBaseValid)
                  00082a29    0000000f     sdl_ex_flash_ecc_test.obj (.text:Flash_getECCTestSingleBitErrorType)
                  00082a38    0000000f     sdl_ex_flash_ecc_test.obj (.text:Flash_setErrorThreshold)
                  00082a47    0000000f     sdl_ex_flash_ecc_test.obj (.text:Interrupt_register)
                  00082a56    0000000e     sdl_ex_flash_ecc_test.obj (.text:Flash_setECCTestAddress)
                  00082a64    0000000e     sdl_ex_flash_ecc_test.obj (.text:Flash_setECCTestECCBits)
                  00082a72    0000000e     driverlib_eabi.lib : interrupt.obj (.text:Interrupt_defaultHandler)
                  00082a80    0000000d     sdl_ex_flash_ecc_test.obj (.text:Flash_disableECCTestMode)
                  00082a8d    0000000d     sdl_ex_flash_ecc_test.obj (.text:Flash_selectLowECCBlock)
                  00082a9a    0000000d     driverlib_eabi.lib : interrupt.obj (.text:Interrupt_disableMaster)
                  00082aa7    0000000d                        : interrupt.obj (.text:Interrupt_enableMaster)
                  00082ab4    0000000d     sdl_ex_flash_ecc_test.obj (.text:SysCtl_clearAllNMIFlags)
                  00082ac1    0000000d     device.obj (.text:SysCtl_setLowSpeedClock)
                  00082ace    0000000d     rts2800_fpu32_eabi.lib : copy_zero_init.c.obj (.text:decompress:ZI:__TI_zero_init_nomemset)
                  00082adb    0000000c     sdl_ex_flash_ecc_test.obj (.text:Flash_clearSingleErrorInterruptFlag)
                  00082ae7    0000000c     sdl_ex_flash_ecc_test.obj (.text:Flash_clearUncorrectableInterruptFlag)
                  00082af3    0000000c     sdl_ex_flash_ecc_test.obj (.text:Flash_disableECC)
                  00082aff    0000000c     sdl_ex_flash_ecc_test.obj (.text:Flash_enableECCTestMode)
                  00082b0b    0000000c     sdl_ex_flash_ecc_test.obj (.text:Flash_performECCCalculation)
                  00082b17    0000000c     sdl_ex_flash_ecc_test.obj (.text:Flash_selectHighECCBlock)
                  00082b23    0000000c     rts2800_fpu32_eabi.lib : args_main.c.obj (.text)
                  00082b2f    0000000b     sdl_ex_flash_ecc_test.obj (.text:Flash_setDataHighECCTest)
                  00082b3a    0000000b     sdl_ex_flash_ecc_test.obj (.text:Flash_setDataLowECCTest)
                  00082b45    0000000b     driverlib_eabi.lib : sysctl.obj (.text:SysCtl_isMCDClockFailureDetected)
                  00082b50    0000000a     sdl_ex_flash_ecc_test.obj (.text:Flash_getECCTestStatus)
                  00082b5a    00000009     sdl_ex_flash_ecc_test.obj (.text:Flash_getErrorCount)
                  00082b63    00000009     rts2800_fpu32_eabi.lib : _lock.c.obj (.text)
                  00082b6c    00000008     sdl_ex_flash_ecc_test.obj (.text:Flash_getTestDataOutHigh)
                  00082b74    00000008     sdl_ex_flash_ecc_test.obj (.text:Flash_getTestDataOutLow)
                  00082b7c    00000008     device.obj (.text:SysCtl_disableWatchdog)
                  00082b84    00000008     sdl_ex_flash_ecc_test.obj (.text:SysCtl_enableNMIGlobalInterrupt)
                  00082b8c    00000008     rts2800_fpu32_eabi.lib : copy_decompress_none.c.obj (.text:decompress:none)
                  00082b94    00000008     f28004x_codestartbranch.obj (.text)
                  00082b9c    00000007     driverlib_eabi.lib : sysctl.obj (.text:SysCtl_resetMCD)
                  00082ba3    00000007     device.obj (.text:__error__)
                  00082baa    00000006     sdl_ex_flash_ecc_test.obj (.text:Interrupt_clearACKGroup)
                  00082bb0    00000003     sdl_ex_flash_ecc_test.obj (.text:SysCtl_getNMIFlagStatus)
                  00082bb3    00000002     driverlib_eabi.lib : interrupt.obj (.text:Interrupt_illegalOperationHandler)
                  00082bb5    00000002                        : interrupt.obj (.text:Interrupt_nmiHandler)
                  00082bb7    00000002     rts2800_fpu32_eabi.lib : pre_init.c.obj (.text)
                  00082bb9    00000001                            : startup.c.obj (.text)

MODULE SUMMARY

       Module                        code   ro data   rw data
       ------                        ----   -------   -------
    .\
       sdl_ex_flash_ecc_test.obj     1037   48        14     
       f28004x_codestartbranch.obj   10     0         0      
    +--+-----------------------------+------+---------+---------+
       Total:                        1047   48        14     
                                                             
    .\device\
       device.obj                    353    0         0      
    +--+-----------------------------+------+---------+---------+
       Total:                        353    0         0      
                                                             
    C:\ti\c2000\C2000Ware_4_01_00_00\driverlib\f28004x\driverlib\ccs\Debug\driverlib_eabi.lib
       sysctl.obj                    1023   154       0      
       flash.obj                     640    155       0      
       gpio.obj                      210    152       0      
       interrupt.obj                 187    0         0      
    +--+-----------------------------+------+---------+---------+
       Total:                        2060   461       0      
                                                             
    C:\ti\ccs1110\ccs\tools\compiler\ti-cgt-c2000_21.6.0.LTS\lib\rts2800_fpu32_eabi.lib
       copy_decompress_lzss.c.obj    49     0         0      
       exit.c.obj                    41     0         6      
       autoinit.c.obj                43     0         0      
       ll_cmp28.asm.obj              30     0         0      
       memcpy.c.obj                  29     0         0      
       ll_aox28.asm.obj              24     0         0      
       boot28.asm.obj                23     0         0      
       _lock.c.obj                   9      0         4      
       copy_zero_init.c.obj          13     0         0      
       args_main.c.obj               12     0         0      
       copy_decompress_none.c.obj    8      0         0      
       pre_init.c.obj                2      0         0      
       startup.c.obj                 1      0         0      
    +--+-----------------------------+------+---------+---------+
       Total:                        284    0         10     
                                                             
       Stack:                        0      0         256    
       Linker Generated:             0      28        0      
    +--+-----------------------------+------+---------+---------+
       Grand Total:                  3744   537       280    


LINKER GENERATED COPY TABLES

__TI_cinit_table @ 00081188 records: 2, size/record: 4, table size: 8
	.data: load addr=00081174, load size=0000000a bytes, run addr=0000a80c, run size=0000000c bytes, compression=lzss
	.bss: load addr=00081184, load size=00000004 bytes, run addr=0000a800, run size=0000000c bytes, compression=zero_init


LINKER GENERATED HANDLER TABLE

__TI_handler_table @ 0008117e records: 3, size/record: 2, table size: 6
	index: 0, handler: __TI_zero_init
	index: 1, handler: __TI_decompress_lzss
	index: 2, handler: __TI_decompress_none


GLOBAL DATA SYMBOLS: SORTED BY DATA PAGE

address     data page           name
--------    ----------------    ----
00000400      10 (00000400)     __stack

0000a800     2a0 (0000a800)     calcECC
0000a801     2a0 (0000a800)     nmiISRFlag
0000a802     2a0 (0000a800)     nmiStatus
0000a803     2a0 (0000a800)     errorISRFlag
0000a804     2a0 (0000a800)     errorStatus
0000a805     2a0 (0000a800)     errorCount
0000a806     2a0 (0000a800)     errorType
0000a808     2a0 (0000a800)     dataOut
0000a80c     2a0 (0000a800)     __TI_enable_exit_profile_output
0000a80e     2a0 (0000a800)     __TI_cleanup_ptr
0000a810     2a0 (0000a800)     __TI_dtors_ptr
0000a812     2a0 (0000a800)     _lock
0000a814     2a0 (0000a800)     _unlock
0000a816     2a0 (0000a800)     result


GLOBAL SYMBOLS: SORTED ALPHABETICALLY BY Name 

page  address   name                           
----  -------   ----                           
0     00082783  C$$EXIT                        
0     00082000  Device_enableAllPeripherals    
0     000825a2  Device_init                    
0     00008000  Flash_initModule               
0     0008261d  GPIO_setAnalogMode             
0     000826c5  GPIO_setDirectionMode          
0     000824c0  GPIO_setPadConfig              
0     00082691  Interrupt_enable               
0     000825e0  Interrupt_initModule           
0     0008283a  Interrupt_initVectorTable      
0     00081172  RamfuncsLoadEnd                
abs   00000172  RamfuncsLoadSize               
0     00081000  RamfuncsLoadStart              
0     00008172  RamfuncsRunEnd                 
abs   00000172  RamfuncsRunSize                
0     00008000  RamfuncsRunStart               
0     0000816e  SysCtl_delay                   
0     000821a7  SysCtl_isPLLValid              
0     00082512  SysCtl_selectOscSource         
0     000827f7  SysCtl_selectXTAL              
0     000828b0  SysCtl_selectXTALSingleEnded   
0     000820e0  SysCtl_setClock                
0     00081188  __TI_CINIT_Base                
0     00081190  __TI_CINIT_Limit               
0     00081190  __TI_CINIT_Warm                
0     0008117e  __TI_Handler_Table_Base        
0     00081184  __TI_Handler_Table_Limit       
1     00000500  __TI_STACK_END                 
abs   00000100  __TI_STACK_SIZE                
0     00082758  __TI_auto_init_nobinit_nopinit 
1     0000a80e  __TI_cleanup_ptr               
0     000826f6  __TI_decompress_lzss           
0     00082b8c  __TI_decompress_none           
1     0000a810  __TI_dtors_ptr                 
1     0000a80c  __TI_enable_exit_profile_output
abs   ffffffff  __TI_pprof_out_hndl            
abs   ffffffff  __TI_prof_data_size            
abs   ffffffff  __TI_prof_data_start           
0     00082ace  __TI_zero_init_nomemset        
0     000828ca  __c28xabi_andll                
0     00082858  __c28xabi_cmpll                
0     0008286a  __c28xabi_cmpull               
0     000828d2  __c28xabi_orll                 
0     000828da  __c28xabi_xorll                
n/a   UNDEFED   __c_args__                     
0     00082ba3  __error__                      
1     00000400  __stack                        
0     00082b23  _args_main                     
0     0008293e  _c_int00                       
1     0000a812  _lock                          
0     00082b6b  _nop                           
0     00082b67  _register_lock                 
0     00082b63  _register_unlock               
0     00082bb9  _system_post_cinit             
0     00082bb7  _system_pre_init               
1     0000a814  _unlock                        
0     00082783  abort                          
1     0000a800  calcECC                        
0     00082267  calculateECC                   
0     00080000  code_start                     
0     0008239c  corrErrorISR                   
1     0000a808  dataOut                        
1     0000a805  errorCount                     
1     0000a803  errorISRFlag                   
1     0000a804  errorStatus                    
1     0000a806  errorType                      
0     00082785  exit                           
0     00082469  main                           
0     00082893  memcpy                         
0     0008255c  nmiISR                         
1     0000a801  nmiISRFlag                     
1     0000a802  nmiStatus                      
1     0000a816  result                         
0     00082409  runCorrectableDataErrorTest    
0     00082658  runCorrectableECCErrorTest     
0     00082727  runUncorrectableErrorTest      
0     00008044  testECCBlock                   


GLOBAL SYMBOLS: SORTED BY Symbol Address 

page  address   name                           
----  -------   ----                           
0     00008000  Flash_initModule               
0     00008000  RamfuncsRunStart               
0     00008044  testECCBlock                   
0     0000816e  SysCtl_delay                   
0     00008172  RamfuncsRunEnd                 
0     00080000  code_start                     
0     00081000  RamfuncsLoadStart              
0     00081172  RamfuncsLoadEnd                
0     0008117e  __TI_Handler_Table_Base        
0     00081184  __TI_Handler_Table_Limit       
0     00081188  __TI_CINIT_Base                
0     00081190  __TI_CINIT_Limit               
0     00081190  __TI_CINIT_Warm                
0     00082000  Device_enableAllPeripherals    
0     000820e0  SysCtl_setClock                
0     000821a7  SysCtl_isPLLValid              
0     00082267  calculateECC                   
0     0008239c  corrErrorISR                   
0     00082409  runCorrectableDataErrorTest    
0     00082469  main                           
0     000824c0  GPIO_setPadConfig              
0     00082512  SysCtl_selectOscSource         
0     0008255c  nmiISR                         
0     000825a2  Device_init                    
0     000825e0  Interrupt_initModule           
0     0008261d  GPIO_setAnalogMode             
0     00082658  runCorrectableECCErrorTest     
0     00082691  Interrupt_enable               
0     000826c5  GPIO_setDirectionMode          
0     000826f6  __TI_decompress_lzss           
0     00082727  runUncorrectableErrorTest      
0     00082758  __TI_auto_init_nobinit_nopinit 
0     00082783  C$$EXIT                        
0     00082783  abort                          
0     00082785  exit                           
0     000827f7  SysCtl_selectXTAL              
0     0008283a  Interrupt_initVectorTable      
0     00082858  __c28xabi_cmpll                
0     0008286a  __c28xabi_cmpull               
0     00082893  memcpy                         
0     000828b0  SysCtl_selectXTALSingleEnded   
0     000828ca  __c28xabi_andll                
0     000828d2  __c28xabi_orll                 
0     000828da  __c28xabi_xorll                
0     0008293e  _c_int00                       
0     00082ace  __TI_zero_init_nomemset        
0     00082b23  _args_main                     
0     00082b63  _register_unlock               
0     00082b67  _register_lock                 
0     00082b6b  _nop                           
0     00082b8c  __TI_decompress_none           
0     00082ba3  __error__                      
0     00082bb7  _system_pre_init               
0     00082bb9  _system_post_cinit             
1     00000400  __stack                        
1     00000500  __TI_STACK_END                 
1     0000a800  calcECC                        
1     0000a801  nmiISRFlag                     
1     0000a802  nmiStatus                      
1     0000a803  errorISRFlag                   
1     0000a804  errorStatus                    
1     0000a805  errorCount                     
1     0000a806  errorType                      
1     0000a808  dataOut                        
1     0000a80c  __TI_enable_exit_profile_output
1     0000a80e  __TI_cleanup_ptr               
1     0000a810  __TI_dtors_ptr                 
1     0000a812  _lock                          
1     0000a814  _unlock                        
1     0000a816  result                         
abs   00000100  __TI_STACK_SIZE                
abs   00000172  RamfuncsLoadSize               
abs   00000172  RamfuncsRunSize                
abs   ffffffff  __TI_pprof_out_hndl            
abs   ffffffff  __TI_prof_data_size            
abs   ffffffff  __TI_prof_data_start           
n/a   UNDEFED   __c_args__                     

[77 symbols]
